:10000000C8C0000054C1000081C10000DFC0000072
:10001000DDC00000DBC00000D9C000002DC1000021
:10002000D5C00000D3C00000D1C00000CFC0000088
:10003000CDC00000F9C10000C9C00000C7C0000069
:10004000E4C10000C3C00000C1C00000BFC0000088
:100050008CC10000A7C10000B9C00000B7C00000FB
:10006000B5C00000B3C00000B1C00000AFC00000C8
:10007000ADC00000ABC00000A9C00000670C680C58
:100080006D0C200C810C970CBE0CCC0C2E0C400C73
:100090006E616E00696E660000407A10F35A00A02F
:1000A000724E18090010A5D4E80000E87648170041
:1000B00000E40B54020000CA9A3B000000E1F50581
:1000C000000080969800000040420F000000A086CB
:1000D00001000000102700000000E80300000000FD
:1000E0006400000000000A000000000001000000A1
:1000F00000002C76D888DC674F0823DFC1DFAE59BB
:10010000E1B1B796E5E3E453C63AE651997696E84D
:10011000E6C28426EB898C9B62ED407C6FFCEFBCD1
:100120009C9F40F2BAA56FA5F490055A2AF75C93FC
:100130006B6CF9676DC11BFCE0E40D47FEF520E632
:10014000B500D0ED902E0300943577050080841E15
:10015000080000204E0A000000C80C333333330F70
:10016000986E12831141EF8D2114893BE65516CF0D
:10017000FEE6DB18D1844B381BF77C1D901DA4BB19
:10018000E424203284725E228100C9F124ECA1E5CE
:100190003D2711241FBECFEFD0E1DEBFCDBF12E05F
:1001A000A0E0B1E0E8ECFCE302C005900D92A23FB4
:1001B000B107D9F726E0A2EFB2E001C01D92A23B41
:1001C000B207E1F70E944A0E0C94621E19CFF89410
:1001D0002091E8053091E9054091E6055091E70549
:1001E000B901641B750BAB014115524081F0F90157
:1001F000F170EA51FC4F80832F5F3F4F3093E90548
:100200002093E8058091C10080628093C1007894BA
:1002100080E090E00895803C28F0E82FF0E0ED5574
:10022000FE4F80810E94861280E090E0089568B1C0
:10023000482F417050E0FA01369621E030E0D901B4
:1002400002C0AA0FBB1FEA95E2F79A2F909596235A
:1002500098B998B14E5F5F4F01C0220F4A95EAF7F7
:10026000292B28B9B3E18B9FF0011124E05EFC4FEC
:1002700080818460808308951F920F920FB60F9241
:1002800011248F9381E08093F70289B182958F705A
:10029000806F803F31F4F894809160008861809392
:1002A00060008F910F900FBE0F901F9018951F92B6
:1002B0000F920FB60F9211248F93AF93BF93EF93CA
:1002C000FF93F89488B1806C88B988B1837F88B92E
:1002D0004498A3E3B3E08C918B7F8C93E0E2F3E04E
:1002E00080818B7F80838C918D7F8C9380818D7FAB
:1002F0008083808188608083FF91EF91BF91AF916F
:100300008F910F900FBE0F901F9018951F920F9214
:100310000FB60F9211248F93AF93BF93EF93FF9378
:10032000F89488B1806C88B988B1837F88B9449883
:10033000E3E3F3E080818B7F8083A0E2B3E08C91E4
:100340008B7F8C9380818D7F80838C918D7F8C932C
:10035000808188608083FF91EF91BF91AF918F91F1
:100360000F900FBE0F901F9018951F920F920FB60F
:100370000F9211248F93EF93FF938091F6028F5F7A
:100380008093F602E091F602F0E08091C600E95019
:10039000FD4F8083FF91EF918F910F900FBE0F90D3
:1003A0001F9018951F920F920FB60F9211242F9342
:1003B0003F938F939F93EF93FF938091E6059091E6
:1003C000E7052091E8053091E90582179307B9F018
:1003D000FC01F170EA51FC4F20812093C600019688
:1003E0009093E7058093E605FF91EF919F918F91A0
:1003F0003F912F910F900FBE0F901F9018958091F5
:10040000C1008F7D8093C100EFCF1F920F920FB676
:100410000F9211248F9381E08093F5028F910F90BA
:100420000FBE0F901F9018951F920F920FB60F924C
:1004300011248F9381E08093F4028F910F900FBE6F
:100440000F901F90189584B7877F84BFE0E6F0E097
:100450008081886180831082E9E6F0E080818A6093
:1004600080838DB383608DBB88B1806D88B987B17F
:100470008C6D87B9599A519A1092C50086E2809383
:10048000C40082E08093C00098E99093C10096E098
:100490009093C20094B1976B94B995B1906B95B954
:1004A00090E59CBD94E09093B8009093BC0084BD0F
:1004B00090E897BD95E095BD80936E009DE0909388
:1004C000810020E034E030938900209388008093FD
:1004D0006F00ECE7F0E08081806C808383E880939C
:1004E0007A008FEF80937E0088E08093680080EF31
:1004F0008093730008950F931F93CF93DF9300D0E1
:1005000000D0CDB7DEB785B1887F866085B92C98DD
:10051000FE0135969E012F5F3F4F9FEF9EBD0DB4AC
:1005200007FEFDCF8EB58293E217F307B9F72C9A39
:100530000A8100933603009323031981612F62958A
:100540006F7070E080E090E00E94571620E030E08D
:1005500048EC50E40E940B1720E030E048E452E4FD
:100560000E94071787FD03C00F5F00932303812FAD
:10057000817011FB992790F9892BD9F5809134036B
:10058000817F8093340380912103817F80932103B5
:100590008B81482F42954F709C81592F5295507FE7
:1005A000252F242B392F32953F7048E03427A9019D
:1005B000585050933803409337035093250340938A
:1005C000240386958695837049E1849FC001112498
:1005D000C29734F02F5F37403093380320933703AE
:1005E0000F900F900F900F90DF91CF911F910F916F
:1005F00008951770110F80913403817F812B8093B0
:10060000340380912103817F182B109321031092D2
:100610003803109237031092250310922403E0CF81
:100620002F923F924F925F926F927F928F929F9202
:10063000AF92BF92CF92DF92EF92FF920F931F93F0
:10064000CF93DF93262F30E040E5649FF001112423
:10065000EA5BFC4F028913890817190780F1E25BF6
:10066000FF4F4081518184179507A8F486E990E0F7
:10067000DF91CF911F910F91FF90EF90DF90CF907E
:10068000BF90AF909F908F907F906F905F904F90B2
:100690003F902F90089540E5649FF0011124E45AA3
:1006A000FC4FC0E003C00081118134968017910790
:1006B00048F4CF5FC031B9F78FEF9FEFD9CF80E01B
:1006C00090E0D6CF1C01D0E07E0181E0E81AF1086D
:1006D00084E1829F6001839FD00C1124EC0CFD1CEF
:1006E000F701EE0FFF1FEE0FFF1FEA5AFC4F60816C
:1006F000718180E090E00E9455164B015C01F7018A
:10070000EE0FFF1FEE0FFF1FEA5BFC4F628973893C
:1007100080E090E00E9455162B013C01CC0DDD1DC0
:10072000CC0FDD1FCC0FDD1FCA5ADC4F68817981E9
:1007300080E090E00E945516A50194010E94531597
:100740006B017C01B10180E090E00E945516A3018D
:1007500092010E9453159B01AC01C701B6010E9492
:100760000B176B017C01B80180E090E00E945516E8
:10077000A30192010E9453159B01AC01C701B60170
:100780000E94BC15A50194010E9454150E942416D4
:10079000CB016ECFCF93DF93E82F80917C00982F11
:1007A000987F8E2F8170892B80937C008BE291E063
:1007B0000197F1F700C000003AE040E050E080917E
:1007C0007A00806480937A0080917A0084FFFCCF65
:1007D000809178002091790090E0922B480F591F6A
:1007E000315069F79A01ADECBCEC0E94E51A969580
:1007F0008795969587959695879523E1E29FE001E9
:100800001124C05EDC4F998788876E2F09DF9F8394
:100810008E83DF91CF910895CF93C82F80917C0074
:100820009C2F91709E5F887F892B80937C008BE248
:1008300091E00197F1F700C0000080917A00806498
:1008400080937A0080917A0084FFFCCF60917800D9
:100850008091790070E0782B80E090E00E9455163E
:100860002AE939E949E150E40E940B170E94291650
:1008700023E1C29FF0011124E05EFC4F7787668779
:10088000CB01CF910895F8948091E8059091E90506
:100890002091E6053091E705AC01421B530B9A010C
:1008A0002115324081F0FC01F170EA51FC4F25E541
:1008B000208301969093E9058093E8058091C1001B
:1008C00080628093C1007894F8948091E8059091BB
:1008D000E9052091E6053091E705BC01621B730B29
:1008E0009B012115324081F0FC01F170EA51FC4F6F
:1008F00025E4208301969093E9058093E805809193
:10090000C10080628093C1007894F8948091E805DA
:100910009091E9052091E6053091E705FC01E21B85
:10092000F30B9F012115324081F0FC01F170EA5177
:10093000FC4F25E8208301969093E9058093E80514
:100940008091C10080628093C1007894ADE3B0E0F3
:100950005FE19D012D50310932BD21BDF89A40B5AE
:10096000F8948091E8059091E9056091E605709111
:10097000E705FC01E61BF70BBF016115724079F03A
:10098000FC01F170EA51FC4F408301969093E90518
:100990008093E8058091C10080628093C1007894C3
:1009A000540F2F5F3F4F2A173B07B1F6D901A05BC9
:1009B000BF4FAD3048E0B40761F6F8948091E80588
:1009C0009091E9052091E6053091E705BC01621B95
:1009D000730B9B012115324079F0FC01F170EA5153
:1009E000FC4F508301969093E9058093E805809130
:1009F000C10080628093C10078941092F302089540
:100A00000F931F93CF93DF9364EA70E081E090E04F
:100A10000E943F1BEC0185E588838091F3028A8365
:100A2000833009F47EC008F47AC0853009F46FC0C1
:100A3000863051F480EA8983E6E4F3E0DE01139620
:100A400001900D928A95E1F750E080E090E08E01F0
:100A50000D551F4FFE01E80FF91F4081F89480915A
:100A6000E8059091E9052091E6053091E705BC0184
:100A7000621B730B9B012115324081F09C01317088
:100A80002A513C4FD9014C9301969093E9058093EC
:100A9000E8058091C10080628093C1007894D801FC
:100AA0004C918081480F4C935F5F298130E02E5F2D
:100AB0003F4F852F90E02817390764F6F89480910E
:100AC000E8059091E9052091E6053091E705FC01E4
:100AD000E21BF30B9F012115324079F0FC01F1700C
:100AE000EA51FC4F408301969093E9058093E80515
:100AF0008091C10080628093C10078941092F302CB
:100B0000CE01DF91CF911F910F910C94F11BBBDEB1
:100B1000CE01DF91CF911F910F910C94F11B19829F
:100B200093CF86E28983E0E2F3E0DE011396019041
:100B30000D928A95E1F788CFF894809160008861E2
:100B400080936000FFCF611126C098B1482F41709B
:100B500050E0BA016A5F7F4F21E030E0F90102C046
:100B6000EE0FFF1F6A95E2F7BF01692B68B998B1D4
:100B70004E5F5F4F01C0220F4A95EAF72095292367
:100B800028B993E1899FF0011124E05EFC4F808138
:100B90008B7F808308954BCBCF92DF92EF92FF92B1
:100BA000CF93DF9390917C00987F282F2170922B18
:100BB00090937C00EBE2F1E03197F1F700C0000088
:100BC00090917A00906490937A0090917A0094FFCB
:100BD000FCCF6091780090917900C82FD0E070E050
:100BE000792B80E090E00E9455162AE037ED43E231
:100BF0005BE30E940B176B017C012DE02C9FC00171
:100C00002D9F900D1124EC01C257D94F2AE43CE0EE
:100C100042E45FE369817A818B819C810E940B179A
:100C20009B01AC01C701B6010E94BC152D813E811C
:100C30004F8158850E945415DF91CF91FF90EF901E
:100C4000DF90CF9008957F928F929F92AF92BF9244
:100C5000CF92DF92EF92FF920F931F93CF93DF9388
:100C6000C82FE82EF12C83E1C89FF0011124E05E2B
:100C7000FC4F7088C188D28840E050E0BA018C2FC8
:100C80000E94321300E010E020E430E440E050E045
:100C9000BA018C2F0E9451138C2F7EDF4B015C0117
:100CA00020E030E040E450E40E94071718160CF4EE
:100CB0006FC02DEC3CEC4CE45DE3C501B4010E9437
:100CC00007171816A4F1D4E014E0672D8C2F0E94AA
:100CD000E3136C2D8C2F0E9412146D2D8C2F0E940B
:100CE000401483E18E9DF0018F9DF00D1124E05E94
:100CF000FC4F9D2F9295990F990F907C80818F7357
:100D0000892B8083D695D69581818E7FD82BD183F0
:100D1000812FDF91CF911F910F91FF90EF90DF9086
:100D2000CF90BF90AF909F908F907F90089520E0DC
:100D300030E040EC5FE3C501B4010E94B81518161D
:100D400014F26FEF8C2F0E94401461E08C2F0E94F0
:100D50005F1487EB9BE00197F1F700C000008C2F38
:100D60001BDF4B015C016D2D8C2F0E94401460E055
:100D70008C2F0E945F142DEC3CEC4CE45EE3C5012B
:100D8000B4010E94B81587FF06C0D2E012E09DCFE3
:100D9000D0E010E09ACFD3E013E097CF2F923F92AC
:100DA0004F925F926F927F928F929F92AF92BF927B
:100DB000CF92DF92EF92FF920F931F93CF93DF9327
:100DC000CDB7DEB764970FB6F894DEBF0FBECDBFC8
:100DD000382E91DB832D37DF232D30E03A872987AA
:100DE00033E1339EF0011124E05EFC4F8081982FA7
:100DF000929596959695937081818170880F880F52
:100E0000892B823041F18081982F92959695969505
:100E1000937081818170880F880F892B8330D9F07E
:100E200080E090E064960FB6F894DEBF0FBECDBFB1
:100E3000DF91CF911F910F91FF90EF90DF90CF90B6
:100E4000BF90AF909F908F907F906F905F904F90EA
:100E50003F902F90089583E169857A85869FA00150
:100E6000879F500D11245A834983FA01EF5DFC4F8F
:100E7000808186958770A1F681E00E94A11200E032
:100E800010E020E430E440E050E0BA01832D0E94FD
:100E9000511340E050E0BA01832D0E9432138FE6D7
:100EA00097E10197F1F700C00000C984DA849FEF51
:100EB000C91AD90AA981BA81A05EBC4FBE83AD838D
:100EC0007D01B6E0EB0EF11CAD80BE80E2E0AE0E1F
:100ED000B11C62E3862E61E0962E0D811E810C5FAF
:100EE0001F4F78E4672E71E0772E05DB60E080E02D
:100EF0000E94C612D70111968C9111978F938C91F5
:100F00008F93F50180811F928F93DF92CF929F92F2
:100F10008F9224E131E03F932F930E94871D61E07F
:100F200080E00E94C612D80111968C9111978F9380
:100F30008C918F937F926F92E4E1F1E0FF93EF93B6
:100F40000E94871DD8014D905C908091220190E015
:100F50000FB6F894DEBF0FBECDBF841595052CF2F9
:100F6000832D1ADE2AE037ED43E25DE30E9454153B
:100F70006D877E87888B9A8B69837B878B83292EED
:100F8000AD81BE818C91982F929596959695937090
:100F900011968C918170880F880F892B1F82823067
:100FA00009F4F4C0832D43D98091230190E0019688
:100FB00043E1E985FA854E9F90014F9F300D112442
:100FC000A901405E5C4F5E834D83DA0114964D911A
:100FD0005C911597841795070CF425C1E12CF12C31
:100FE0004D815E815C8B4B8B4A015EE0850E911CCE
:100FF000B9016F5D7C4F7E836D83CB88DC8874E0A4
:10100000C70ED11C8DE0A985BA858A9F80018B9F70
:10101000100D11240956194F4BE7A42E41E0B42EB0
:1010200054E1652E51E0752E83C065DAAB89BC8929
:101030008C91982F929596959695937011968C9188
:101040008170880F880F892B09F4E7C0EB89FC8930
:101050008081982F92959695969593708181817055
:10106000880F880F892B843009F4D7C0AD81BE81E9
:101070008C918695877009F0D0C0BFEFEB1AFB0A00
:10108000EDE2EE16E1E0FE0668F0D6018D919C914E
:101090009C0124193509253031050CF47CC32C0141
:1010A000E12CF12C60E080E00E94C612F8018381FF
:1010B0008F9382818F9381818F9380818F931F92F1
:1010C0001F921F921F922F92FB81FF932B852F93CC
:1010D00039813F93BF92AF927F926F920E94871D9A
:1010E00061E080E00E94C612D60111968C911197A2
:1010F0008F938C918F93F40181818F9380818F9353
:1011000022E931E03F932F937F926F920E94871DD7
:101110008091230190E001960FB6F894DEBF0FBED8
:10112000CDBFD6012D913C91821793070CF47BC063
:10113000832D72DB853C994008F072CEEB89FC89E7
:101140008081982F92959695969593708181817064
:10115000880F880F892B823009F067CFD4018D91D9
:101160009C918D3DB5E09B0708F047C0883E9340B9
:1011700008F05BCFEF81EF5FEF836E2F832D0E942E
:10118000401461E0832D0E945F144FCF83E12985D5
:101190003A85829FF001839FF00D1124E25DFC4FA0
:1011A000FE83ED8310E001C0122F612F832D0E947A
:1011B000401461E0832D0E945F14832D38D887EBA3
:1011C0009BE00197F1F700C00000832D25DB60E074
:1011D000832DB9DC60E0832D0E945F1421E0210F94
:1011E000AD81BE818D919C91883E9340E8F21F8332
:1011F00061E0832D0E945F14D5CEEF81E150EF8333
:101200006E2F832D0E94401461E0832D0E945F1495
:10121000D4018D919C91AACF3D84832D0E94BE1450
:101220008FEF9FEFFFCD60E0832D8DDC60E0832D9D
:101230000E945F14EFE6F7E13197F1F700C000007C
:10124000832DAADC962E872E782E692E2AE037ED84
:1012500043E25CE3D401F3016B2F7A2F8F2F9E2F93
:101260000E940717181684F42AE037ED43E25CE386
:10127000D401F3016B2F7A2F8F2F9E2F0E945315CD
:10128000962E872E782E692E5D854E8598898A89BF
:10129000052F142F292F382FF401C3014F2F582D5C
:1012A000692F762D832D0E945113B0912301BD83A8
:1012B000E0912201EF83BE1708F4A1C223E1E98582
:1012C000FA852E9FC0012F9F900D11249C01205E56
:1012D0003C4F38872F8389010C5F1F4F790138E01D
:1012E000E30EF11CA4EACA2EA1E0DA2EB8EB4B2ED5
:1012F000B1E05B2E24E12E9FA0012F9F500D112401
:101300005F874E87BC016F5D7C4F798B688B3D8614
:10131000372C722C262C6B847D81A72EB12CD80102
:101320008D919C918A159B05E4F1E5D860E080E001
:101330000E94C612D70111968C9111978F938C91B0
:101340008F937F92BB81BF936F92E981EF93DF927E
:10135000CF9224E131E03F932F930E94871D61E0FB
:1013600080E00E94C612D80111968C9111978F933C
:101370008C918F932F923F928F929F925F924F9278
:10138000E4E1F1E0FF93EF930E94871D0FB6F8941C
:10139000DEBF0FBECDBFD8018D919C918A159B05F4
:1013A00024F68D85F7D98DECBD81B89F812D112450
:1013B000869586958695EE85FF85E80FF11DCF0110
:1013C000EE0FFF1FEE0FFF1FEA5AFC4FB182A08203
:1013D000880F991F880F991FFC01EA5BFC4FD7010A
:1013E0008D919C91938B828BEF81F8858081982FD2
:1013F000929596959695937081818170880F880F4C
:10140000892B09F409CF8081982F9295969596950E
:10141000937081818170880F880F892B843009F443
:10142000FBCEA889B9898C918695877009F0F4CE96
:10143000BD81BA50BD8380912201B81708F06CCFEE
:101440008F833D84209023018DEC289E212D112433
:10145000269526952695EF81E89F812D1124869566
:101460008695869510E00DEC94E149855A85949F08
:101470007001959FF00C1124B701680F711DAB012D
:10148000440F551F440F551FDA01A85ABC4FBA83A9
:10149000A983FA01EA5AFC4FFC83EB83C701820F50
:1014A000911D9C01220F331F220F331FA901485A9F
:1014B0005C4F5E834D83B9016A5A7C4F7C876B8792
:1014C0002D863E861701109F812D112486958695C5
:1014D0008695D101A80FB11DB98BA88BFD01EE0F28
:1014E000FF1FEE0FFF1FEA5AFC4F812F90E0918300
:1014F0008083E981FA816081718180E090E00E94BF
:1015000055166B017C01AB81BC816D917C9180E0B3
:1015100090E00E9455164B015C01E889F989EE0FB5
:10152000FF1FEE0FFF1FEA5BFC4FF98BE88BAD81CD
:10153000BE816D917C9180E090E00E945516A701DC
:1015400096010E9453152B013C01612F70E080E051
:1015500090E00E945516A50194010E9453159B012D
:10156000AC01C301B2010E940B172B013C01EB85BA
:10157000FC856081718180E090E00E945516A50194
:1015800094010E9453159B01AC01C301B2010E945A
:10159000BC15A70196010E9454150E942916A8891E
:1015A000B98953967C936E935297165FBF811B1730
:1015B00008F489CF2D843E841AE0120D103A08F009
:1015C000B4C08DEC289E912D1124969596959695F4
:1015D000BF81B89F812D11248695869586950DEC47
:1015E00024E1E985FA852E9F70012F9FF00C1124CC
:1015F0009701280F311DA901440F551F440F551F96
:10160000BA01685A7C4F7A836983DA01AA5ABC4FBF
:10161000BC83AB83F701E90FF11D9F01220F331F3C
:10162000220F331FA901485A5C4F5E834D83B901D5
:101630006A5A7C4F7C876B873F821701109F812DF0
:101640001124869586958695D101A80FB11DBF8777
:10165000AE87FD01EE0FFF1FEE0FFF1FEA5AFC4F92
:10166000812F90E091838083E981FA81608171818B
:1016700080E090E00E9455166B017C01AB81BC813B
:101680006D917C9180E090E00E9455164B015C01C9
:10169000EE85FF85EE0FFF1FEE0FFF1FEA5BFC4F8D
:1016A000FF87EE87AD81BE816D917C9180E090E0F7
:1016B0000E945516A70196010E9453152B013C016B
:1016C000612F70E080E090E00E945516A501940122
:1016D0000E9453159B01AC01C301B2010E940B177C
:1016E0002B013C01EB85FC856081718180E090E0FD
:1016F0000E945516A50194010E9453159B01AC014F
:10170000C301B2010E94BC15A70196010E945415A5
:101710000E942916AE85BF8553967C936E9352978F
:10172000165F103A08F48ACF3F8020E5E985FA85F4
:101730002E9FC0012F9F900D1124895B9C4FDC01CF
:101740002C91222309F454C080E529853A85829F93
:10175000F001839FF00D1124EA5BFC4F83E1829F2F
:10176000D001839FB00D1124A05EBC4F12968C91C6
:101770001297808350968C915097858751968C91C3
:101780005197868752968C918787832D0E940115E9
:1017900081E0D7D645CB60E0832DD5D960E0832D9D
:1017A0000E945F1460E080E0F1D624E131E040E186
:1017B00050E061E070E089E591E00E94D21D61E0B7
:1017C00080E0E4D624E131E040E150E061E070E007
:1017D0008AE691E00E94D21D832D0E94BE141092D1
:1017E000F7028091F7028823E1F38FEF9FEF1ACB86
:1017F0004CE050E06CEC71E00E946D1DA5CFBF8104
:101800002D80BB2309F4D8CE1FCECF93DF93C09198
:10181000EC05CC1FCC27CC1F8091EC058F778093F3
:10182000EC0581E08093F302E091EC058E2F90E0CF
:101830008A30910580F4FC01E25CFF4F0C94DF1AC2
:101840008091ED0593E1C99FE0011124C05EDC4F5A
:1018500090E09B878A87DF91CF91089583E1C89FAD
:10186000E0011124C05EDC4F888182958370823054
:1018700091F79091ED05888190FB82F98883EBCFF9
:101880008091ED05837093E1C99FF0011124E05E22
:10189000FC4F982F9295907F80818F7C892B80833D
:1018A0008091EE05809322018091EF0580932301C2
:1018B000808182958370823009F47CC0808182951A
:1018C0008370813041F68C2FDF91CF9167CA34D974
:1018D0008091ED058093F302BECF9091ED0583E1F9
:1018E000C89FF0011124E05EFC4F808190FB81F9DC
:1018F000808360E08C2F27D960E08C2FDF91CF911F
:10190000DEC78091ED0593E1C99FF0011124E05EEF
:10191000FC4F808B8091EE05818B6091ED058C2FC3
:1019200052D76091EE058C2FDF91CF917BC78C2F22
:1019300090E02091ED0533E1389FF001399FF00DE3
:101940001124E05EFC4F228B2DE0289FE001299FAF
:10195000D00D1124C257D94F6091320370E080E05E
:1019600090E00E9455162BE734E14EEC51E40E94C2
:10197000BC1569877A878B879C876DCF8091ED0531
:1019800093E1C99FF0011124E05EFC4F82838C2F0C
:10199000F5D7DF91CF91CEC74091EB0550E06DEECA
:1019A00075E086E493E00E945D1D8C2FDF91CF915E
:1019B0000C9401158C2FDF91CF9172C0DF92EF92C2
:1019C000FF920F931F93CF93DF930091F6020023B2
:1019D00009F45EC0015010E00F5F1F4FC0E0D0E07F
:1019E00082E0E82EDD24D39493E0F92E17C08130F5
:1019F00008F43FC0823031F59093EC0580918D065C
:101A0000980F90938D06F092F2028091F602815029
:101A10008093F6022196C017D107D1F1FE01E8505C
:101A2000FD4F90818091F202813009F7943668F57C
:101A30009093EB0580918D06980F90938D06E09220
:101A4000F202E3CF2091EB05482F50E030E02E5F0B
:101A50003F4F24173507A4F0FA01E951FA4F938359
:101A600020918D06920F90938D068F5F8093F202E6
:101A7000CCCF953551F690938D06D092F202C5CF1A
:101A800080918D06981301C0C0DE1092F202BDCF86
:101A9000DF91CF911F910F91FF90EF90DF9008950C
:101AA000EF92FF920F931F93CF93DF93C82F81E0A4
:101AB00048D560E080E06AD524E131E040E150E0C3
:101AC00061E070E084ED91E00E94D21DEC2EF12CDB
:101AD00023E1C29F80011124F801E05EFC4F808168
:101AE000982F929596959695937081818170880F25
:101AF000880F892BD0E0823009F45EC083E18E9D8F
:101B000080018F9D100D1124005E1C4FF801808113
:101B1000829583708230A9F58091F602811146C0CA
:101B20008091F30281113FC0F801808182FF33C0B0
:101B30008081982F9295969596959370818181706A
:101B4000880F880F892B823099F18C2F0E94170102
:101B500087EB9BE00197F1F700C000008C2F0E94FB
:101B60000C04813D974090F2D1506D2F8C2F88D678
:101B700061E08C2FA4D6F801808182958370823039
:101B800059F280818B7F8083DF91CF911F910F91DC
:101B9000FF90EF90089560E08C2F0E94A30560E015
:101BA0008C2F8DD6B3CF0E940005BECF07DFB8CFF4
:101BB00061E08C2F84D6C9CF8F01025F1F4F01C017
:101BC000D22F6D2F8C2F5CD661E08C2F78D68C2F86
:101BD0000E94170187EB9BE00197F1F700C000001E
:101BE0008C2F0E940C0460E08C2F0E94A30560E003
:101BF0008C2F65D621E02D0FF80180819181883EE0
:101C00009340F0F27BCFFF920F931F93CF93DF931C
:101C10008FE59AEE0197F1F700C0000060E080E0E8
:101C2000B5D48FEF73D461E08FE0B0D48FEF6ED472
:101C300010E0C1E0DFEF0FE08FEDF82E89B1829563
:101C40008F70806F8F3FE9F08FE59AEE0197F1F783
:101C500000C0000060E08C2F99D48D2F57D461E034
:101C6000802F8C1B93D48D2F51D4CF5FC03131F78F
:101C7000DF251F5FC0E089B182958F70806F8F3F35
:101C800019F7123008F381E0DF91CF911F910F9186
:101C9000FF9057C4CF93DF9300D000D0CDB7DEB70D
:101CA00061E070E083E090E00E943F1B4C0186E21F
:101CB000E0E2F3E0DF011D928A95E9F78AE1EEE8C0
:101CC000F6E0DF011D928A95E9F780EAE6E4F3E0A9
:101CD000DF011D928A95E9F7809120038E7F809322
:101CE00020038091330381608093330381E08093EC
:101CF0009B0689E190E090933E0380933D0390938F
:101D00002B0380932A0386E091E09093AF068093A3
:101D1000AE060E9423026FD476DFE2D580E02ED695
:101D200081E02CD680E00E94230681E00E942306F9
:101D300078940E94000511E01B8277E0272E72E064
:101D4000372EB981BC838091F60281119EC08091AB
:101D5000F302811166C08091200383FD68C08091E9
:101D6000330383FD64C08091F502811190C080919E
:101D7000F402882341F01092F402113009F42DC1CD
:101D8000133009F42AC28091F7028823E1F28FE52B
:101D90009AEE0197F1F700C000001092F70289B1A6
:101DA00082958F7080958F70942D9295907F982B4F
:101DB000882309F4D7C09C8160FA90F950FA91F910
:101DC00070FA92F997709983902F990F990F990F44
:101DD000A981A92BAC83A2FDDFC0113009F0B3CFDC
:101DE000823009F4D9C208F4C6C2833009F4ECC2C7
:101DF000843009F0E4C2D4018C9190E0019663E054
:101E000070E00E94CC1AF4018083882309F4EEC2AA
:101E1000D40111961C9284E0482E512C66246394C0
:101E200092CF0E9400058091200383FF98CF60E04D
:101E300080E0ACD324E131E040E150E061E070E0CB
:101E400085EE91E00E94D21D61E080E09FD324E105
:101E500031E044E050E061E070E086EF91E00E9404
:101E6000D21D80E053D324E131E04BE050E061E04B
:101E700070E08BEF91E00E94D21D89B182958F7046
:101E8000806F873FD1F70E949C0598DD60CF10924C
:101E9000F5020E947B02E12CF12CDE2C8E2D0E949B
:101EA0000C04853C994058F023E12E9DF0012F9DB4
:101EB000F00D1124E05EFC4F80818D7F808360E017
:101EC0008D2D0E94A30560E08D2DF9D487EB9BE05A
:101ED0000197F1F700C000008D2D0E9423068D2D83
:101EE0000E94CA0393E19E9DF0019F9DF00D112475
:101EF000E05EFC4F8081982F929596959695937011
:101F000081818170880F880F892B61F480818D7F9A
:101F10008083AFEFEA1AFA0AB2E0EB16F10409F097
:101F2000BCCF25CF8081982F9295969596959370EA
:101F300081818170880F880F892B8430D1F1808155
:101F400081FF08C086819781228533858217930798
:101F500008F474C160E08D2DB2D460E08D2D0E9434
:101F6000A305D7CFBC8160FAB0F950FAB1F970FA85
:101F7000B2F9000F000F000FB770B02BBC83B2FD99
:101F800026C0907F903809F474C100E0712C55246C
:101F90005394612C11E0D7CE843009F45BC108F46E
:101FA00037C1883009F0CFCE81E0CBD2412C10E090
:101FB000CACE808181FFD1CF8481958122853385EE
:101FC0008217930750F68D2D0E941701A2CF00E0D3
:101FD000712C55245394612CB6CE60E080E0D6D2AB
:101FE000EB81AE2EB12CF3E1FA9D6001FB9DD00C8C
:101FF00011249601205E3C4F3A832983D901129621
:102000008C911F928F93C50101969F938F933F925E
:102010002F9254E1E52E51E0F52EFF92EF920E94AF
:10202000871DF601EF5DFC4F8081869587700FB6A6
:10203000F894DEBF0FBECDBF09F0F5C0A981BA810B
:1020400015968C9115978F9314968C918F93EBE343
:10205000F2E0FF93EF93FF92EF920E94871D0F90A3
:102060000F900F900F900F900F9033E13A9DF00179
:102070003B9DF00D1124E05EFC4F8081982F9295DE
:1020800096959695937081818170880F880F892B22
:10209000823009F451C108F0D5C0882309F4E6C0A4
:1020A000813011F487E032D261E080E06FD2A3E1A9
:1020B000AA9DC001AB9D900D1124FC01E05EFC4F78
:1020C0007F0183858F9382858F932DE132E03F934B
:1020D0002F9344E1C42E41E0D42EDF92CF920E9490
:1020E000871DD7018C91982F929596959695937010
:1020F00011968C9111978170880F880F892B0F9002
:102100000F900F900F900F900F9009F4CBC08C910F
:10211000982F929596959695937011968C918170C3
:10212000880F880F892B813009F4BCC0F7018081AA
:10213000982F929596959695937081818170880FCE
:10214000880F892B843009F4FAC0F70187818F93B7
:1021500086818F9328E332E03F932F93DF92CF92D3
:102160000E94871D0F900F900F900F900F900F906F
:1021700093E19A9DF0019B9DF00D1124E05EFC4FD0
:10218000808181FF9DC0808182FF97C089EDBED193
:10219000D4018C91813009F496C0823009F4B0C02A
:1021A000FC8160FAF0F950FAF1F970FAF2F9F7707F
:1021B000802F880F880F880FF82BFC838F2F857056
:1021C000813009F0E0CD0F5F0F710C3009F0DBCDED
:1021D0008093F70277247394D6CD60E080E0D6D167
:1021E00024E131E040E150E061E070E081E492E020
:1021F0000E94D21D61E080E0C9D124E131E040E1DC
:1022000050E061E070E082E592E00E94D21DBBCD1B
:102210008150823008F097CD81E08093F702015E13
:102220000F71712C90CD24E131E044E050E061E089
:1022300070E088E192E00E94D21D17CF61E08D2D01
:102240003ED3C1CE833079F0843009F02DCF84E0C5
:102250005DD12ACFD4011C928B810E94CE0600E072
:10226000712C612C70CD83E051D11ECF86E04ED110
:102270001BCFB3E12B81B29FF0011124E05EFC4F34
:10228000808181FB992790F981E08927908180FBEB
:1022900091F9908360E0822F12D360E08B810E94DD
:1022A000A30573CE24E131E047E050E061E070E047
:1022B00087E292E00E94D21D5BCF8AED27D168CFE2
:1022C0008DE224D165CF11968C911197982F937040
:1022D00091F4893208F081C061E083E057D124E1B4
:1022E00031E043E050E061E070E086E691E00E947A
:1022F000D21DF40181818F5FD40111968C9350CF50
:10230000F4018181982F937099F4893208F06AC0A2
:1023100060E084E03BD124E131E042E050E061E064
:1023200070E087E691E00E94D21DD40111968C9155
:102330008F5FF401818334CF85E0E8D0B5CE668528
:10234000778580E090E0B1D420E030E04AE754E4C3
:1023500013D49F938F937F936F932FE232E03F9339
:102360002F93DF92CF920E94871D0FB6F894DEBFA5
:102370000FBECDBFFDCE813011F5F40111838081F8
:102380008130B1F1823009F464C044244394512C6B
:10239000662463941B82D7CCD40111961C931197A9
:1023A0008C91813009F43DC0823009F468C062E04C
:1023B000462E512C66246394E1E0EB83C4CC482E76
:1023C000512C66246394BFCC81E0BBD093E0492EAE
:1023D000512C6624639413E0B6CC1C9211961C9287
:1023E000A9D27ACF10821182A5D292CFA3D210CDDA
:1023F00023E13B81239FF0011124E05EFC4F8285A5
:10240000938521E030E0009711F420E030E0821B5A
:10241000930B9387828744244394512C66246394BE
:1024200092CCB3E12B81B29FF0011124E05EFC4F0E
:102430008285938521E030E086399105A9F1820FEC
:10244000931F9387828732E0432E512C6624639436
:102450007ACC83E19B81899FF0011124E05EFC4FDF
:10246000828191E0811101C090E0891B82838B8180
:1024700085D244244394512C6624639464CC33E184
:102480008B81389FF0011124E05EFC4F828191E046
:10249000883169F0890F82838B8170D222E0422ECD
:1024A000512C662463944FCC20E030E0C8CF90E0FC
:1024B000F1CFF8949091BC00906A9093BC009091F9
:1024C000BC0097FFFCCF9EE49093BB009091BC00B2
:1024D0009F7D9093BC009091BC0090689093BC004D
:1024E0009091BC0097FFFCCF8093BB008091BC0013
:1024F00080688093BC008091BC0087FFFCCF8091F6
:10250000BC0080698093BC0078940895CF93DF93DA
:10251000C82FD82FD07F8D2F8560CBDF8D2F816086
:10252000C8DF80E1C89FE00111248C2F8560C1DFE6
:102530008C2F8160BEDF80E18A95F1F7DF91CF912A
:102540000895CF93DF93C82FD82FD07F8D2F84602D
:10255000B0DF8D2FAEDF20E1C29FC0011124846067
:10256000A8DF8C2F8295807FA4DFC13031F098E204
:102570009A95F1F7DF91CF9108958FE496E4019752
:10258000F1F700C00000DF91CF91089561708F7066
:1025900090E4699F800D11248068D3CFCF92DF92A1
:1025A000FF920F931F93CF93DF9384EAC82E82E0AC
:1025B000D82EF12CD0E08F2D8064C3DF8601C8E0D7
:1025C00003C0F801D1918F018D2FA0DFC150C9F751
:1025D000F8E0FF0E80E4F81631F0F601D781F8E05C
:1025E000CF0ED11CE8CFDF91CF911F910F91FF90BB
:1025F000DF90CF900895CF9380E05BDF2FEB84EDE9
:1026000091E0215080409040E1F700C00000C5E01B
:1026100084E04FDF80E04DDFC150D1F728EC2A95F0
:10262000F1F784E246DF80E244DF8AE28ADF88E075
:1026300088DF81E086DF86E084DF8CE082DFCF9177
:10264000ADCF95B1987F6770692B65B92C9891E1F2
:102650009EBD0DB407FEFDCF8EBD0DB407FEFDCFB0
:102660002C9A0895CF92DF92EF92FF92CF93DF934F
:102670006A017B01C82FC1702BE734E14EEC51E4B5
:10268000C701B601C8D3E5D2D62F64E06C0F8D2FF9
:10269000D8DF8D2FDF91CF91FF90EF90DF90CF901B
:1026A00008958F929F92AF92BF92CF92DF92EF9256
:1026B000FF920F931F93CF93DF93E82F4A015B01A3
:1026C000C901B801CE2ED12C2E2F2170C22FCC0FD4
:1026D000A5019401E8D19B01AC0163E373E383E5B9
:1026E00090E44AD222E03BE247E051E494D322E76F
:1026F0003AE84EE051E4D7D1ACD2D62F61E06C0F6E
:102700008D2F9FDF83E18C9D80018D9D100D112405
:10271000005E1C4FF801D08B2AE43CE042E45FE30A
:10272000C501B40178D320E030E04FE753E473D320
:1027300025E33EE542E050E41FD28BD2D62F6C2F2A
:102740008D2F7FDFF801D18B2DE02C9DC0012D9DB9
:10275000900D11249C012257394F7901608970E056
:1027600080E090E0A2D222E73AE84EE051E49CD12A
:1027700022E03BE247E051E4FFD1F701618372833D
:10278000838394836D2F70E080E090E08ED225E308
:102790003EE542E050E43FD320E030E04FE753E431
:1027A000EBD1F7016583768387839087DF91CF91A3
:1027B0001F910F91FF90EF90DF90CF90BF90AF905F
:1027C0009F908F9008951F93CF93DF93C82F162F5C
:1027D000682F6170660F6F5F812F33DF83E1C89FC1
:1027E000F0011124E05EFC4F108B8DE0C89FE001EA
:1027F0001124C257D94F612F70E080E090E055D28C
:1028000022E73AE84EE051E44FD122E03BE247E0D4
:1028100051E4B2D169837A838B839C83DF91CF911A
:102820001F9108951F93CF93DF93C82F162F682F02
:102830006170660F812F05DF83E1C89FF0011124CD
:10284000E05EFC4F118B8DE0C89FE0011124C25760
:10285000D94F612F70E080E090E027D225E33EE57C
:1028600042E050E4D8D220E030E04FE753E484D196
:102870006D837E838F839887DF91CF911F91089519
:10288000CF93DF9393E1899FF0011124E05EFC4F29
:10289000628B9DE0899FE0011124C257D94F70E0FF
:1028A00080E090E002D22BE734E14EEC51E464D1B9
:1028B00069877A878B879C87DF91CF910895962FC0
:1028C000682F61706C5F23E1829FF0011124E05E4C
:1028D000FC4F892F81709289899F802D1124B1CE60
:1028E00021E080E090E092BD81BDF89A823081F0D5
:1028F0008330C1F030B5813091F030932203243021
:10290000C1F001962F5F92BD81BDF89A823081F7A8
:1029100040B550E050932B0340932A03F2CF3093FD
:102920003503EFCF80B590E090933E0380933D0355
:1029300008950895F89480E090E092BD81BD8230C2
:10294000C9F0833099F0813069F02091220320BDD5
:10295000FA9AF99AF999FECF01968430910569F7B0
:10296000789408952091350320BDF2CF20913D0346
:1029700020BDEECF20912A0320BDEACF0F931F93F5
:10298000CF93DF93C82F20E5829FF0011124EA5BEB
:10299000FC4F80E090E04C2F50E063E1C69FD001F7
:1029A0001124AE5DBC4F2C91BC01D0E52D9F600D74
:1029B000711D11249B01205D3F4F32BD21BDF89A4E
:1029C00020B5219301968035910569F780E5849FB4
:1029D0008001859F100D11240A5B1C4FF80165854D
:1029E0008C2FF1DEF80166858C2F1CDFF8016785DE
:1029F0008C2F46DF60E08C2FDF91CF911F910F91DC
:102A00005ECFCF92DF92EF92FF920F931F93CF93FF
:102A1000DF93082FF89481E094DD60E080E0B6DD7C
:102A200024E231E04DE050E061E070E083EE92E0BE
:102A30000E94D21D61E080E0A9DD20E5029F8001B7
:102A400011240A5B1C4FC0E0D0E0680185E0E82E4D
:102A5000F12CF60180819E0140E5849F200D311DFF
:102A60001124C901C09692BD81BDF80181918F01E9
:102A7000219680BDFA9AF99AF999FECFCE01B70155
:102A80008BD5892B69F0C035D10519F77894DF9182
:102A9000CF911F910F91FF90EF90DF90CF9008950D
:102AA0008FEF34DDF0CF5058BB27AA270ED075C169
:102AB00066D130F06BD120F031F49F3F11F41EF459
:102AC0005BC10EF4E095E7FB51C1E92F77D180F3AC
:102AD000BA17620773078407950718F071F49EF51B
:102AE0008FC10EF4E0950B2EBA2FA02D0B01B9016A
:102AF00090010C01CA01A0011124FF27591B99F074
:102B0000593F50F4503E68F11A16F040A22F232F7F
:102B1000342F4427585FF3CF469537952795A795CF
:102B2000F0405395C9F77EF41F16BA0B620B730B76
:102B3000840BBAF09150A1F0FF0FBB1F661F771FE7
:102B4000881FC2F70EC0BA0F621F731F841F48F49C
:102B5000879577956795B795F7959E3F08F0B3CF22
:102B60009395880F08F09927EE0F9795879508950C
:102B7000D9D008F481E008950CD00FC107D140F0FE
:102B8000FED030F021F45F3F19F0F0C0511139C18F
:102B9000F3C014D198F39923C9F35523B1F3951BCE
:102BA000550BBB27AA2762177307840738F09F5F6E
:102BB0005F4F220F331F441FAA1FA9F333D00E2EDD
:102BC0003AF0E0E830D091505040E695001CCAF74A
:102BD00029D0FE2F27D0660F771F881FBB1F26170F
:102BE00037074807AB07B0E809F0BB0B802DBF01E2
:102BF000FF2793585F4F2AF09E3F510568F0B6C0FB
:102C000000C15F3FECF3983EDCF3869577956795BE
:102C1000B795F7959F5FC9F7880F911D9695879592
:102C200097F90895E1E0660F771F881FBB1F6217B1
:102C300073078407BA0720F0621B730B840BBA0B6F
:102C4000EE1F88F7E095089504D06894B111D9C0BB
:102C50000895BCD088F09F5790F0B92F9927B751AD
:102C6000A0F0D1F0660F771F881F991F1AF0BA9550
:102C7000C9F712C0B13081F0C3D0B1E00895C0C02F
:102C8000672F782F8827B85F39F0B93FCCF3869546
:102C900077956795B395D9F73EF4909580957095A3
:102CA00061957F4F8F4F9F4F0895E89409C097FB20
:102CB0003EF490958095709561957F4F8F4F9F4F13
:102CC0009923A9F0F92F96E9BB279395F695879557
:102CD00077956795B795F111F8CFFAF4BB0F11F41A
:102CE00060FF1BC06F5F7F4F8F4F9F4F16C08823C1
:102CF00011F096E911C0772321F09EE8872F762FF7
:102D000005C0662371F096E8862F70E060E02AF037
:102D10009A95660F771F881FDAF7880F9695879523
:102D200097F90895990F0008550FAA0BE0E8FEEFF8
:102D300016161706E807F907C0F012161306E4077F
:102D4000F50798F0621B730B840B950B39F40A2678
:102D500061F0232B242B252B21F408950A2609F456
:102D6000A140A6958FEF811D811D089597F99F675A
:102D700080E870E060E008959FEF80EC0895002403
:102D80000A941616170618060906089500240A94D0
:102D900012161306140605060895092E0394000C56
:102DA00011F4882352F0BB0F40F4BF2B11F460FFE5
:102DB00004C06F5F7F4F8F4F9F4F089557FD90580E
:102DC000440F551F59F05F3F71F04795880F97FBEF
:102DD000991F61F09F3F79F08795089512161306A9
:102DE0001406551FF2CF4695F1DF08C016161706D8
:102DF0001806991FF1CF869571056105089408950D
:102E0000E894BB2766277727CB0197F908958ADFD7
:102E100008F48FEF08950BD0C0CFB1DF28F0B6DFF4
:102E200018F0952309F0A2CFA7CF1124EACFC6DF6F
:102E3000A0F3959FD1F3950F50E0551F629FF001CD
:102E4000729FBB27F00DB11D639FAA27F00DB11D26
:102E5000AA1F649F6627B00DA11D661F829F2227AF
:102E6000B00DA11D621F739FB00DA11D621F839F36
:102E7000A00D611D221F749F3327A00D611D231F0C
:102E8000849F600D211D822F762F6A2F11249F575A
:102E900050408AF0E1F088234AF0EE0FFF1FBB1F7D
:102EA000661F771F881F91505040A9F79E3F51051C
:102EB00070F05CCFA6CF5F3FECF3983EDCF38695D5
:102EC00077956795B795F795E7959F5FC1F7FE2BC7
:102ED000880F911D9695879597F90895A0E1B0E028
:102EE000E3E7F7E181C37C011B016A01FC01178262
:102EF0001682838181FF2AC39E012F5F3F4F3901D4
:102F0000F7019381F10193FD859193FF81911F0159
:102F1000882309F417C3853239F493FD859193FF13
:102F200081911F01853231F4B70190E0FFD5560140
:102F30006501E6CF10E0512C912CFFE1F915D8F096
:102F40008B3279F038F4803279F08332A1F4F92DA4
:102F5000F0612EC08D3261F0803369F4292D21603B
:102F60002DC0392D3260932E892D8460982E2AC071
:102F7000E92DE86015C097FC2DC020ED280F2A3000
:102F800088F496FE06C03AE0139F200D1124122FFC
:102F900019C08AE0589E200D1124522EE92DE062BE
:102FA0009E2E10C08E3231F496FCCCC2F92DF06406
:102FB0009F2E08C08C3621F4292D2068922E02C045
:102FC000883641F4F10193FD859193FF81911F01B2
:102FD0008111B3CF9BEB980F933020F4992D906122
:102FE000805E07C09BE9980F933008F059C1992D76
:102FF0009F7E96FF16E09F73992E853619F4906494
:10300000992E08C0863621F4392F3068932E02C0DD
:103010001111115097FE07C01C3350F444244394FF
:10302000410E27E00BC0183038F027E017E005C04C
:1030300027E09CE3492E02C0212F412C560184E059
:10304000A80EB11CF6016081718182819381042DEB
:10305000A30150D46C01F981FC87F0FF02C0F3FF9B
:1030600006C091FC06C092FE06C000E205C00DE25B
:1030700003C00BE201C000E08C858C7019F00111D7
:1030800043C280C297FE10C04C0CFC85F4FF04C004
:103090008A81813309F44A94141474F528E02415C4
:1030A00078F588E0482E2CC096FC2AC0812F90E04D
:1030B0008C159D059CF03CEFC3163FEFD30674F0D2
:1030C000892D8068982E0AC0E2E0F0E0EC0FFD1F29
:1030D000E10FF11D8081803319F411501111F4CFEB
:1030E00097FE0EC044244394410E812F90E0C816F1
:1030F000D9062CF41C1904C04424439401C010E0E8
:1031000097FE06C01C141D0434F4C601019605C0C8
:1031100085E090E002C081E090E00111019611236A
:1031200031F0212F30E02F5F3F4F820F931F252D6D
:1031300030E08217930714F4581A01C0512C892DDE
:10314000897041F4552031F0B70180E290E0EED46F
:103150005A94F8CF002321F0B701802F90E0E6D4F5
:1031600093FC08C0552031F0B70180E390E0DED435
:103170005A94F8CF97FE4AC04601D7FE02C0812C70
:10318000912CC60188199909F301E80FF91FFE87F0
:10319000ED87960124193109388B2F87012F10E014
:1031A0001195019511093FEF8316930621F4B7019C
:1031B0008EE290E0BBD4C814D9044CF08F85988976
:1031C0008815990524F4ED85FE85818101C080E391
:1031D000F1E08F1A91082D853E852F5F3F4F3E8786
:1031E0002D878016910624F0B70190E09FD4DBCFA5
:1031F000C814D90441F49A81963320F4953319F414
:103200003C8534FF81E3B70190E048C08A81813377
:1032100019F09C859F7E9C87B70190E087D411119F
:1032200005C094FC16C085E690E015C0B7018EE29B
:1032300090E07CD41E5F82E001E0080FF301E80F0C
:10324000F11D8081B70190E071D4802F0113F4CF7C
:10325000E8CF85E490E0B70169D4D7FC06C0C1147B
:10326000D10441F4EC85E4FF05C0D194C194D108A8
:103270008DE201C08BE2B70190E058D480E32AE0F0
:10328000C216D1042CF08F5FFAE0CF1AD108F7CF25
:10329000B70190E04BD4B701C601C09647D449C1ED
:1032A000833631F0833779F0833509F052C01FC07F
:1032B000560132E0A30EB11CF6018081898301E042
:1032C00010E0630111C05601F2E0AF0EB11CF6012F
:1032D000C080D18096FE03C0612F70E002C06FEF06
:1032E0007FEFC60109D48C01F92DFF7713C0560179
:1032F00022E0A20EB11CF601C080D18096FE03C070
:10330000612F70E002C06FEF7FEFC601CBD38C015D
:10331000F92DF0689F2EF3FD18C0852D90E0081759
:10332000190798F4B70180E290E000D45A94F5CFE1
:10333000F60197FC859197FE81916F01B70190E0AE
:10334000F5D351105A94015011090115110581F757
:10335000F0C0843611F0893659F5560197FE09C040
:1033600024E0A20EB11CF6016081718182819381FB
:103370000AC0F2E0AF0EB11CF60160817181072E28
:10338000000C880B990BF92DFF769F2E97FF09C033
:1033900090958095709561957F4F8F4F9F4FF06806
:1033A0009F2E2AE030E0A3012FD4C82EC6183EC0BD
:1033B000092D853721F40F7E2AE030E01DC0097FFA
:1033C0008F3691F018F4883559F0BCC0803719F069
:1033D000883711F0B7C0006104FF09C0046007C05E
:1033E00094FE08C0066006C028E030E005C020E179
:1033F00030E002C020E132E0560107FF09C084E05E
:10340000A80EB11CF601608171818281938108C090
:10341000F2E0AF0EB11CF6016081718180E090E0B6
:10342000A301F2D3C82EC6180F77902E96FE0BC0BC
:10343000092D0E7FC11650F494FE0AC092FC08C0FC
:10344000092D0E7E05C0DC2C092D03C0DC2C01C02B
:10345000D12E04FF0DC0FE01EC0DF11D80818033E3
:1034600011F4097E09C002FF06C0D394D39404C0AE
:10347000802F867809F0D39403FD10C000FF06C0AA
:103480001C2DD51478F4150D1D190CC0D51450F44D
:10349000B70180E290E04AD3D394F8CFD51410F46A
:1034A0005D1801C0512C04FF0FC0B70180E390E00C
:1034B0003DD302FF16C001FD03C088E790E002C0C3
:1034C00088E590E0B7010CC0802F867851F001FFAD
:1034D00002C08BE201C080E207FD8DE2B70190E0FF
:1034E00025D3C11630F4B70180E390E01FD311500B
:1034F000F8CFCA94F301EC0DF11D8081B70190E083
:1035000015D3C110F6CF15C0F4E0F51550F584E0E1
:10351000581A93FE1EC0011125C02C8523FF27C019
:1035200000E910E0392D3071932EF801849181115A
:1035300021C0552009F4FCCCB70180E290E0F6D21E
:103540005A94F7CFF7018681978123C08FEF9FEFC1
:1035500020C0B70180E290E0E9D25A945110F9CF2F
:10356000DACF512CB701802F90E0E0D2D6CF04E91A
:1035700010E0D8CF91108052B70190E0D7D20F5F02
:103580001F4FD3CF23E0251510F483E0C1CF512C7A
:10359000C4CF6096E2E144C097FB072E16F4009476
:1035A00006D077FD08D057D007FC05D03EF49095A3
:1035B00081959F4F0895709561957F4F0895EE0F07
:1035C000FF1F0590F491E02D0994A29FB001B39FD5
:1035D000C001A39F700D811D1124911DB29F700D1C
:1035E000811D1124911D08952F923F924F925F9259
:1035F0006F927F928F929F92AF92BF92CF92DF9203
:10360000EF92FF920F931F93CF93DF93CDB7DEB767
:10361000CA1BDB0B0FB6F894DEBF0FBECDBF0994FB
:103620002A88398848885F846E847D848C849B8452
:10363000AA84B984C884DF80EE80FD800C811B8160
:10364000AA81B981CE0FD11D0FB6F894DEBF0FBE8F
:10365000CDBFED010895AA1BBB1B51E107C0AA1FF6
:10366000BB1FA617B70710F0A61BB70B881F991F23
:103670005A95A9F780959095BC01CD0108950F93B7
:103680001F93CF93DF93869F8001879F100D969F96
:10369000100D1124C8010DD0EC01009721F0A801F4
:1036A00060E070E013D2CE01DF91CF911F910F91B6
:1036B00008950F931F93CF93DF938230910510F4F9
:1036C00082E090E0E091AA06F091AB0620E030E0C5
:1036D000A0E0B0E0309719F140815181028113815F
:1036E00048175907C8F08417950769F4109731F007
:1036F00012960C93129713961C9327C00093AA0658
:103700001093AB0622C02115310519F0421753075B
:1037100018F49A01BD01EF01DF01F801DBCF21159B
:103720003105F9F0281B390B2430310580F48A81EA
:103730009B816115710521F0FB019383828304C095
:103740009093AB068093AA06FE01329644C0FE0118
:10375000E20FF31F8193919322503109398328831B
:103760003AC02091A8063091A906232B41F420915C
:103770000201309103013093A9062093A8062091FD
:103780000001309101012115310541F42DB73EB7FB
:103790004091040150910501241B350BE091A806CE
:1037A000F091A906E217F307A0F42E1B3F0B281790
:1037B000390778F0AC014E5F5F4F2417350748F0AA
:1037C0004E0F5F1F5093A9064093A80681939193D3
:1037D00002C0E0E0F0E0CF01DF91CF911F910F91A7
:1037E0000895CF93DF93009709F481C0FC013297CD
:1037F00013821282A091AA06B091AB06109781F4B1
:1038000020813181820F931F2091A8063091A90653
:103810002817390751F5F093A906E093A80667C069
:10382000ED0120E030E0CE17DF0740F44A815B81F4
:103830009E0141155105F1F0EA01F5CFD383C28312
:1038400040815181840F951FC817D90759F4888189
:103850009981840F951F0296918380838A819B8131
:10386000938382832115310529F4F093AB06E0930D
:10387000AA063DC0E901FB83EA8349915991C40F2F
:10388000D51FEC17FD0761F480819181840F951F8E
:103890000296E90199838883828193819B838A833D
:1038A000E0E0F0E012968D919C911397009719F04B
:1038B000FD01DC01F7CF8D919C9111979D012E5F49
:1038C0003F4F820F931F2091A8063091A906281719
:1038D000390769F4309729F41092AB061092AA06C2
:1038E00002C013821282B093A906A093A806DF91AA
:1038F000CF910895283008F027E03327DA01990F97
:10390000311D87FD916000966105710539F43260C3
:103910002E5F3D9330E32A95E1F708959F3F30F005
:1039200080387105610509F03C5F3C5F3D93913043
:1039300008F08068911DDF93CF931F930F93FF9240
:10394000EF92192F987F9695E92F96959695E90F06
:10395000FF27EE50FF4F99273327EE24FF24A701BE
:10396000E70105900894079428F4360FE71EF81E27
:10397000491F511D660F771F881F991F0694A1F7D5
:103980000590079428F4E70EF81E491F561FC11D25
:10399000770F881F991F661F0694A1F7059007945B
:1039A00028F4F80E491F561FC71FD11D880F991FF5
:1039B000661F771F0694A1F70590079420F4490F1E
:1039C000561FC71FD81F990F661F771F881F0694A1
:1039D000A9F784911095177041F0D695C795579522
:1039E0004795F794E7941A95C1F7E8E9F0E06894F1
:1039F0001590159135916591959105907FE273959C
:103A0000E118F10A430B560BC90BD009C0F7E10CC2
:103A1000F11E431F561FC91FD01D7EF4703311F4D1
:103A20008A95E6CFE894015030F0080F0AF4002799
:103A3000021708F4202F2395022F7A3328F079E318
:103A40007D932A95E9F710C07D932A9589F606940F
:103A500097956795379517951794E118F10A430BD9
:103A6000560BC90BD00998F023957E9173957A3344
:103A700008F070E37C932013B8F77E9170617D931A
:103A800030F0839571E37D9370E32A95E1F711247B
:103A9000EF90FF900F911F91CF91DF91992787FDB4
:103AA00090950895FC010590615070400110D8F781
:103AB000809590958E0F9F1F0895FB01DC0102C039
:103AC00001900D9241505040D8F70895DC0101C09B
:103AD0006D9341505040E0F70895FB01DC014150E7
:103AE000504048F001900D920020C9F701C01D928E
:103AF00041505040E0F70895FC0161507040019042
:103B00000110D8F7809590958E0F9F1F0895A0E023
:103B1000B0E0ECE8FDE178CDAE01475F5F4F6F812B
:103B200078858D819E81DAD9E2E08ACD0F931F934B
:103B3000CF93DF93FB01238121FD03C08FEF9FEF24
:103B40002CC022FF16C0468157812481358142173F
:103B5000530744F4A081B1819D012F5F3F4F318312
:103B600020838C93268137812F5F3F4F37832683B5
:103B700014C08B01EC01FB010084F185E02D099557
:103B8000892BE1F6D80116968D919C911797019695
:103B900017969C938E931697CE01DF91CF911F912C
:103BA0000F910895A0E0B0E0E7EDFDE123CD5B01CA
:103BB0004A017901D90113962C9121FF1DC0C0E063
:103BC000D0E0C815D905D9F08C016C01CA0CDB1CFA
:103BD000C8010C151D0571F00F5F1F4FD701189616
:103BE000ED91FC911997B701DC018C910995892B16
:103BF00079F305C02196E5CF80E090E001C0CE01C9
:103C0000CDB7DEB7ECE012CDFA01AA27283051F18A
:103C1000203181F1E8946F936E7F6E5F7F4F8F4FFD
:103C20009F4FAF4FB1E03ED0B4E03CD0670F781F5C
:103C3000891F9A1FA11D680F791F8A1F911DA11D41
:103C40006A0F711D811D911DA11D20D009F468947A
:103C50003F912AE0269F11243019305D3193DEF622
:103C6000CF010895462F4770405D4193B3E00FD0D8
:103C7000C9F7F6CF462F4F70405D4A3318F0495DC3
:103C800031FD4052419302D0A9F7EACFB4E0A695A6
:103C90009795879577956795BA95C9F700976105C8
:103CA000710508959B01AC010A2E0694579547951E
:103CB00037952795BA95C9F7620F731F841F951F13
:083CC000A01D0895F894FFCF48
:103CC8000000B20620000000000200000000E7002B
:103CD8000000000000000002000000000B010000CE
:103CE8000000288200000002000000000B01000014
:103CF80000004B252E31752050252E327520546D2D
:103D08003D252E3375202D0043414C49422E205429
:103D1800633D252E3375202D00CDE5E4EEF1F2E06C
:103D2800F2EEF7EDFBE920202000F2E5EFEBEEE202
:103D3800EEE920EAEEEDF2E0EAF2002530342E3228
:103D4800662D2530342E326620473D2530342E32FC
:103D58006600493D252E34756D412054633D252E5E
:103D68003375200056483D2530342E326620446D88
:103D78003D252E3375202D00564C3D2530342E32EE
:103D8800662054633D252E3375202D004445464159
:103D9800554C5400D0D3D7CD2E20CAC0CBC8C1D0E3
:103DA800CEC2CAC000C7C0D9C8D2C020CFCE20D288
:103DB800CECAD3212100CDC0C62E0020C4CBDF201F
:103DC800D1C1D0CED1C0004B252E31752023252E50
:103DD8003275202054EF3D002D2D2D200054F33D49
:103DE800252E3375012000CED2CACBDED72E00494E
:103DF8003D25342E32664100D2ED3D252E33640137
:103E080000D3CACD2D322030392E30392E32303100
:103E18003900CDE0E3E0E5E220C0EBE5EAF1E0EDD2
:103E2800E4F00041A042A1E045A3A4A5A64BA74DFC
:103E3800484FA8504354A9AA58E1ABACE2ADAE62D2
:103E4800AFB0B161B2B3B4E365B6B7B8B9BABBBC89
:103E5800BD6FBE7063BF79E478E5C0C1E6C2C3C474
:103E6800C5C6C7000E1F1F1F0E000008140800005B
:103E780000000000040A111111111104041F040AA2
:103E8800111F04040E0A0A0A0A0E04030A080B0A80
:103E9800081B0208080402010808080808040402AC
:103EA8000F0A08D1CED5D0C0CDC5CDC8C52E2E2E6F
:023EB800000008
:00000001FF
